:020000001428C2
:08000800F000030E8301F1007A
:100010000A08F2008A01942972088A00710E83008E
:10002000F00E700E0B110900830185018601870116
:1000300094019801831606309F000030850000303F
:1000400086000030870088308100831220308400D1
:100050008001840A841F2828AE0AAF0A81018B011F
:100060000B118B168B17EA2008210D210030282157
:100070000230D000D1010330D200D301E0214C087E
:10008000B5004D08B400AE21122117218E218E211A
:100090006330D000D101C930D200D301E0214C0837
:1000A000B5004D08B400AE21122117218E218E21FA
:1000B0003B30D0000130D1002B30D2000130D300D2
:1000C000E0214C08B5004D08B400AE2112211721E3
:1000D0008E218E210C30D400D5010330D600D701FB
:1000E000FB215808B5005908B400AE211221172190
:1000F0008E218E21E830D400FD30D5008830D60026
:100100001330D700FB215808B5005908B400AE21C0
:10011000122117218E218E210C30D400D5010330FD
:10012000D600D701FB215808B5005908B400AE210C
:10013000122117218E218E216430D400D501213067
:10014000D600D701FB215808B5005908B400AE21EC
:10015000122117218E218E215A08B5005B08B400A8
:10016000AE21122117218E218E212508B5002608E7
:10017000B400AE211221172101302E02031DC32825
:100180005E218E21E22802302E02031DCA2864213E
:100190008E21E22803302E02031DD12866218E21F4
:1001A000E22804302E02031DD82869218E21E2287E
:1001B00005302E02031DE0286D218E21AE01E228BC
:1001C0007A218E213C302B02031CE928AE0AAB01B8
:1001D000AF0AB5288221033037210330372103309D
:1001E00037210230372102303721083037210030E3
:1001F00037210830372100303721013037210030D6
:10020000372106303721003037210C3037210800E4
:100210000030372101303721822908303721003062
:10022000372182290A3037210830372182293608C0
:1002300022213708222138082221390822213A08B0
:1002400022210800303EB000300E482130084829F5
:10025000B30018308A0033080020B20001308A0051
:100260003208003E031908002321B30A29290F3957
:10027000B100003085000000000031088700000058
:100280000000203085000000000000308500822939
:100290000F39B100103085000000000031088700E0
:1002A00000000000303085000000000010308500A4
:1002B00000000000003085007C2908001030870015
:1002C00088210030870088295E215E295E215E2119
:1002D0005E295E215E215E215E295E215E215E2116
:1002E0005E215E296D215E296D2164296D216629BB
:1002F0006D2169296D216D29A70104302702031C96
:100300007D290800A70111302702031C832908005A
:10031000A80105302802031C89290800A8012830FB
:100320002802031C8F290800A00AA70AA10AAD30E1
:100330002102031CAD29A101A30AA80AA90AAA0A3D
:10034000A20A14302202031CAD29A201A40AA50AA4
:100350000319A60AAB0AAC0AAD0A0C28340E0F39F1
:10036000F03EB700B707E23EB800323EBA003408AC
:100370000F39B807B807BA07E93EB900B907B90796
:10038000350E0F39B907BA07B90DBA0DBA09BA0D4A
:1003900035080F39BA07B70D0730B6000A30BA076B
:1003A000B903031CCF29B907B803031CD329B80725
:1003B000B703031CD729B707B603031CDB29003496
:1003C0005008CC005108CD00CE01CF01CB01103038
:1003D0004B02031CEC2908004C1CF4295208CE07E0
:1003E0000318CF0A5308CF07CF0CCE0CCD0CCC0C82
:1003F0004B08CB0AE7295408D8005508D900DA0180
:10040000DB010310D80DD90DDA0DDB0DCB01103057
:100410004B02031C0F2A0310DB0CDA0C08005708F0
:10042000DB025608DA02031CDB03DB1F1F2A560817
:10043000DA070318DB0A5708DB070310202A031426
:0E044000D80DD90DDA0DDB0D4B08CB0A072ABB
:1030000082077734313436342034653400347734F1
:0A3010006F3472346C346434003401
:02400E00B13FC0
:00000001FF
